:10E0000031400003B240805A20013F4002000F938C
:10E0100005242F839F4FE8E50002FB233F400300C8
:10E020000F9304241F83CF430202FC233040B4E14A
:10E03000304034E0001332C2D24266000402A2D360
:10E04000020232D200130F1232C2E2B323000224C2
:10E0500092D30202C243230032D23F4100130E4347
:10E060000E9F132C03430343034303430343034320
:10E070000343034303430343034303430343034370
:10E08000034303431E530E9FED2B3041B240805A91
:10E090002001F24005002100C2432900F24219008C
:10E0A000C2432600C2432E00F24030001B00F24063
:10E0B000F9FF2200F2432A00F240DBFF1A00E2439C
:10E0C0002400C2432C00E2432500C2432D00D2426B
:10E0D000FD105700D242FC105600F24020005300C1
:10E0E0003041D2D36100F24080FF6100F240450030
:10E0F0006200C2436300E2426400D2C36100D2D333
:10E10000010030414E4FE2B30300FD27C24E6700CD
:10E1100030410B120A120912094F4A4E4B434B9ED3
:10E12000082C4F4B0F596F4FB01204E15B534B9AC1
:10E13000F82B39413A413B4130411B5B33326D286A
:10E140003131352E322D382D3120584F4E2F584F2A
:10E15000464629204543484F204F46460D0A004772
:10E16000696E676572205465726D696E616C2052CC
:10E17000656164790D0A1B5B33306D0050434C00C0
:10E180007265626F6F74006563686F206F6E004523
:10E1900063686F206973204F4E0D0A006563686FD6
:10E1A000206F6666004563686F206973204F46469E
:10E1B0000D0A0000314060020B430943B0128CE0AD
:10E1C000F2C219003E404F000F41CF4300001F53E1
:10E1D0001E83FB233E404F000A413A5050000F4A35
:10E1E000CF4300001F531E83FB23B012E2E03F40E9
:10E1F000FF00B0125EE03F43B0125EE03F43B0125A
:10E200005EE07F400D00B01204E17F400A00B012D2
:10E2100004E17E4024003F403AE1B01212E17E402A
:10E220001C003F405FE1B01212E182430202C24390
:10E230002B00C2432300F2D2190032D27F401100DA
:10E24000B01204E192B3020225247F401300B01201
:10E2500004E132C2F2C219000F4AB0129CE34E4FE1
:10E260008E11E2C3230092C302020F410F5EFF40F2
:10E270000D004F000F4E0F51FF400A0050001E537B
:10E280000F4AB01212E132D27F401100B01204E105
:10E29000F2D21900A2B202022B247F401300B01266
:10E2A00004E132C2A2C202023D4003000E413F40DF
:10E2B0007CE1B01238E50F9364203E4080E10F41CD
:10E2C000B01268E50F9359203E4087E10F41B0122C
:10E2D00068E50F9343247E400C003F408FE1B0126D
:10E2E00012E119430B4332D27F401100B01204E116
:10E2F000A2B30202A72732C2A2C302025E420402F4
:10E300007E921D247E900D0005240F4B0F51CF4EA1
:10E3100000001B533B903D000F2CF2900D000402B7
:10E3200009241993022432D28D3F5F420402B012B5
:10E3300004E1F93F0B93F527A2D20202F23F0F4B03
:10E340000F51CF4300000B9301243B537F42B01287
:10E3500004E17F402000B01204E1DC3F3E409CE13C
:10E360000F41B01268E50F93BD277E400D003F407E
:10E37000A5E1B01212E10943B53FB240085A2001AD
:10E38000FF3F4F4B5F534E4F0F41B01260E4E2C36B
:10E390002300A83F3150A0003040E6E50B120A12DE
:10E3A0000912094F4D430B430C43E2C22200E2B372
:10E3B00020000B241B530C633B9020A103203C90B6
:10E3C00007003F24E2B32000F523D2C32100B2406E
:10E3D000085A20013E424D5DE2B22000FD23E2B327
:10E3E00020004F434F634DDFD2D32100E2B2200023
:10E3F000FD27D2C321003E53EE234A4D0C430B4A66
:10E400003B530C9B222CB240085A20013E424D5DEA
:10E41000E2B22000FD23E2B320004F434F634DDF03
:10E42000D2D32100E2B22000FD27D2C321003E5307
:10E43000EE230F490F5CCF4D00001C530C9BE32BC8
:10E44000043CB240085A2001FF3FD2D32100B24021
:10E45000805A20014F4A8F1139413A413B413041A6
:10E460000B120A120A4F0C430D43E2B320000220A4
:10E470000F435F3CE2D22200D2C32100E2B320006E
:10E480000B241C530D633C9020A103203D900700FA
:10E490004C24E2B32000F523B240085A20014D4E2F
:10E4A0003C42E2B32000FD234F4D4F5F4F434F6F7F
:10E4B000C2DF2100E2C22100E2B32000FD27E2D248
:10E4C0002100D2C321004D5D3C53EB234B4E0E4344
:10E4D0001B932124B240085A20010F4A0F5E6D4F52
:10E4E0003C42E2B32000FD234F4D4F5F4F434F6F3F
:10E4F000C2DF2100E2C22100E2B32000FD27E2D208
:10E500002100D2C321004D5D3C53EB231E530F4B22
:10E510003F530E9FDF2BE2C22200F2D00500210004
:10E52000B240805A20011F43043CB240085A2001E7
:10E53000B03F3A413B4130410B120B4D0D930A2441
:10E540000C4F0D4E6E4D1D536F4C1C534F9E0420AF
:10E550003B53F8230C43053C5C4CFFFF5F4DFFFF32
:10E560000C8F0F4C3B4130410B120A12091208125A
:10E570000B4F0A4E694E1A5349931524084A1883C3
:10E580001853C8930000FC23088A6F4B1B534F930A
:10E590000C244F99FA230D480E4A0F4BB012B6E5E2
:10E5A0000F93F3233B530F4B013C0F433841394149
:10E5B0003A413B4130410B120B4F0D9302200D436A
:10E5C0000F3C6F4E1E536C4B4C9F06201B534C93BD
:10E5D000F6273D53F623F33F4D4C5F4EFFFF0D8F63
:08E5E0000F4D3B413041FF3FAC
:02E5E800000031
:10FFE00030E030E046E030E030E030E030E036E075
:10FFF00030E030E030E030E030E030E030E000E0B1
:040000030000E00019
:00000001FF
